:100000000C9436000C94BE090C945E000C945E00B7
:100010000C945E000C945E000C945E000C945E00E8
:100020000C945E000C945E000C945E000C94FD0A2F
:100030000C945E000C945E000C945E000C945E00C8
:100040000C945E000C945E000C945E000C945E00B8
:100050000C945E000C945E000C945E000C945E00A8
:100060000C945E000C945E00C806ED0911241FBEBE
:10007000CFEFD8E0DEBFCDBF11E0A0E0B1E0E4EA11
:10008000F6E102C005900D92A030B107D9F721E04A
:10009000A0E0B1E001C01D92AB32B207E1F710E081
:1000A000CCE6D0E004C02297FE010E944C0BC8367B
:1000B000D107C9F70E943F0B0C94500B0C94000021
:1000C0008A3091054CF020E030E02F5F3F4F0A97D7
:1000D0008A309105D4F702C020E030E022953295B5
:1000E000307F3227207F3227822B932B08950E9466
:1000F000220B529887B18F7C87B984B1887F84B9ED
:1001000087B1876087B988B1887F88B984B18863EF
:1001100084B985B1877C85B98DE091E00E94B00AF1
:10012000803829F460E08DE091E00E94C80A0895CB
:100130008DE091E00E94B80A90E0BC016295729552
:10014000707F7627607F762795958795959587951B
:100150009595879595958795682B40E083E091E08C
:100160000E9409078DE091E00E94B40A90E0BC0172
:1001700062957295707F7627607F76279595879533
:10018000959587959595879595958795682B40E0EA
:1001900083E091E00E9409078DE091E00E94B00A9F
:1001A00090E0BC0162957295707F7627607F76271C
:1001B0009595879595958795959587959595879527
:1001C000682B40E083E091E00E94090783E091E022
:1001D0000E949C0708958DE091E00E94BC0A90E087
:1001E000BC0162957295707F7627607F7627959522
:1001F0008795959587959595879595958795682B7E
:1002000040E083E091E00E9409078DE091E00E94C8
:10021000C00A90E0BC0162957295707F7627607F7E
:100220007627959587959595879595958795959535
:100230008795682B40E083E091E00E9409078DE0FC
:1002400091E00E94C40A90E0BC0162957295707FB3
:100250007627607F762795958795959587959595CF
:10026000879595958795682B40E083E091E00E9403
:10027000090783E091E00E949C0708958DE091E0DA
:100280000E94B00A0E94980008950196662309F41E
:10029000C8C08230910509F446C08330910509F445
:1002A00081C0019709F084C140E06FEF83E091E0E5
:1002B0000E9409078DE091E00E94C00A90E0BC0115
:1002C00062957295707F7627607F762795958795E2
:1002D000959587959595879595958795682B40E099
:1002E00083E091E00E9409078DE091E00E94C40A3A
:1002F00090E0BC0162957295707F7627607F7627CB
:1003000095958795959587959595879595958795D5
:10031000682B40E083E091E00E94090783E091E0D0
:100320000E949C0708958DE091E00E94BC0A90E035
:10033000BC0162957295707F7627607F76279595D0
:100340008795959587959595879595958795682B2C
:1003500040E083E091E00E94090740E06FEF83E016
:1003600091E00E9409078DE091E00E94C40A90E0AC
:10037000BC0162957295707F7627607F7627959590
:100380008795959587959595879595958795682BEC
:1003900040E083E091E00E94090783E091E00E9441
:1003A0009C0708958DE091E00E94BC0A90E0BC019A
:1003B00062957295707F7627607F762795958795F1
:1003C000959587959595879595958795682B40E0A8
:1003D00083E091E00E9409078DE091E00E94C00A4D
:1003E00090E0BC0162957295707F7627607F7627DA
:1003F00095958795959587959595879595958795E5
:10040000682B40E083E091E00E94090740E06FEF35
:1004100083E091E00E94090783E091E00E949C073D
:1004200008958230910509F446C08330910509F49E
:1004300081C0019709F0BCC040E06FEF83E091E01C
:100440000E9409078DE091E00E94B40A90E0BC018F
:1004500062957295707F7627607F76279595879550
:10046000959587959595879595958795682B40E007
:1004700083E091E00E9409078DE091E00E94B00ABC
:1004800090E0BC0162957295707F7627607F762739
:100490009595879595958795959587959595879544
:1004A000682B40E083E091E00E94090783E091E03F
:1004B0000E949C0708958DE091E00E94B80A90E0A8
:1004C000BC0162957295707F7627607F762795953F
:1004D0008795959587959595879595958795682B9B
:1004E00040E083E091E00E94090740E06FEF83E085
:1004F00091E00E9409078DE091E00E94B00A90E02F
:10050000BC0162957295707F7627607F76279595FE
:100510008795959587959595879595958795682B5A
:1005200040E083E091E00E94090783E091E00E94AF
:100530009C0708958DE091E00E94B80A90E0BC010C
:1005400062957295707F7627607F7627959587955F
:10055000959587959595879595958795682B40E016
:1005600083E091E00E9409078DE091E00E94B40AC7
:1005700090E0BC0162957295707F7627607F762748
:100580009595879595958795959587959595879553
:10059000682B40E083E091E00E94090740E06FEFA4
:1005A00083E091E00E94090783E091E00E949C07AC
:1005B00008950E94360B809302011A9B03C088EEB7
:1005C00093E003C0813CF9F4FACF1A9949C040C0C6
:1005D00083B1109201011092000183B18873885F8A
:1005E000893320F485FF03C02D9A02C080E02D9846
:1005F00084FF02C02C9A01C02C9883FF02C02B9A62
:1006000008952B980895199B03C088EE93E004C0C9
:10061000803C09F03FC0F9CF19992CC034C083B198
:10062000109201011092000183B183B18873885048
:1006300085FF02C02D9A01C02D9884FF02C02C9A1C
:1006400001C02C9883FF02C02B9A08952B9808951F
:100650008091000190910101892B09F4B9CFB9CFA4
:10066000EFE9FFE03197F1F700C000000197009734
:1006700079F3ABCFEFE9FFE03197F1F700C000006D
:100680000197009749F68091000190910101892B13
:1006900031F2C6CF0895BF92CF92DF92EF92FF92D0
:1006A0000F931F93CF93DF93189B95C2189BAEC1F6
:1006B0008FE99FE00197F1F700C000001899F8CF8B
:1006C000A5C10F5F1F4F083C110514F000E010E0BA
:1006D000189B0BC0189B08C0EFE9FFE03197F1F7BA
:1006E00000C000001899F8CF2196C330D10509F455
:1006F0006CC03CF4C130D10579F0C230D10509F1AC
:1007000077C1C530D10509F4EAC00CF4A5C0C630E4
:10071000D10509F426C16CC10536110534F060E03D
:1007200082E090E00E94450102C00E9498001A9960
:1007300002C0199B44C260E08DE091E00E94C80AAB
:100740003EC20536110534F060E081E090E00E9481
:10075000450102C00E9498001A9B13C08E2D9F2D48
:100760001A9975C16AC1807F60E1680F02C061E0BB
:10077000680F603608F060E08DE091E00E94CE0ADC
:100780001EC2199B1CC28E2D9F2D199973C169C160
:1007900082958F70682F70E0615071096295729533
:1007A000707F7627607F7627696004C0882329F0F0
:1007B0006FEF680F613618F403C069E501C069E5A1
:1007C0008DE091E00E94CE0AFAC10536110534F0A1
:1007D00060E080E090E00E94450102C00E94980025
:1007E0001A9B17C08E2D9F2D1A9958C14DC1807F1D
:1007F00060E1680F08C0833228F49F5F807F692F13
:10080000682B01C060E040E08DE091E00E94D40AD6
:10081000D6C1199BD4C18E2D9F2D199951C148C1A4
:10082000982F9F7069F482958F7090E00197829560
:100830009295907F9827807F9827682F696006C0DF
:100840009150807F692F682B01C063E240E08DE00A
:1008500091E00E94D40AB3C140980536110534F0E6
:100860006D2D80E090E00E94450102C00E94EB00E7
:100870001A9B15C08E2D9F2D1A9936C12BC1807FD2
:1008800060E1680F04C09F5F807F692F682B62332F
:1008900008F060E08DE091E00E94E00A90C1199BB1
:1008A0008EC18E2D9F2D199932C128C182958F70CE
:1008B00090E0019782959295907F9827807F982766
:1008C000682F696004C09150807F692F682B611187
:1008D00001C061E38DE091E00E94E00A70C105363D
:1008E000110534F06D2D81E090E00E94450102C0B9
:1008F0000E94EB001A9B15C08E2D9F2D1A991BC1CB
:1009000010C1807F60E1680F04C09F5F807F692F06
:10091000682B633108F06D2D8DE091E00E94E60AAE
:100920004EC1199B4CC18E2D9F2D199917C10DC118
:1009300082958F7090E0019782959295907F98278D
:10094000807F9827682F696004C09150807F692F4D
:10095000682B611101C06C2D8DE091E00E94E60AC8
:100960002EC10536110534F06D2D82E090E00E9415
:10097000450102C00E94EB001A9B15C08E2D9F2DD1
:100980001A99F6C0FFC0807F60E1680F04C09F5FC6
:10099000807F692F682B6A3908F060E08DE091E074
:1009A0000E94EC0A0CC1199B0AC18E2D9F2D19992A
:1009B000FCC0F2C08823A1F082958F7090E001976F
:1009C00082959295907F9827807F9827682F6960FD
:1009D0000AC0882339F09150807F692F682B03C0AB
:1009E0006B2D01C06B2D8DE091E00E94EC0AE7C0F9
:1009F00088B1887F88B98FE99FE00197F1F700C03F
:100A00000000C730D1050CF0E6C05BCEC1E0D0E0FD
:100A100000E010E00F2EF8EEEF2EF02D0F2EF3E099
:100A2000FF2EF02D0F2EF2E1CF2EF02DDD24D394EA
:100A30000F2EF9E9BF2EF02D4BCE8DE091E00E94F4
:100A4000B40A982F9F70993009F091CE8CCEEFE9BF
:100A5000FFE03197F1F700C000000197009769F3BC
:100A60007FCE8DE091E00E94B40A982F9F7009F428
:100A70008FCE9CCEEFE9FFE03197F1F700C0000088
:100A80000197009771F381CE8DE091E00E94B80A42
:100A9000982F9F70993009F0AECEA9CEEFE9FFE014
:100AA0003197F1F700C000000197009769F39CCEE1
:100AB0008DE091E00E94B80A882309F4C6CEB0CE3A
:100AC000EFE9FFE03197F1F700C0000001970097D0
:100AD00079F3A3CE8DE091E00E94BC0A982F9F701D
:100AE000993009F0D0CECBCEEFE9FFE03197F1F7A6
:100AF00000C000000197009769F3BECE8DE091E041
:100B00000E94BC0A982F9F7009F4D0CEDCCEEFE98A
:100B1000FFE03197F1F700C000000197009771F3F3
:100B2000C2CE8DE091E00E94C00A982F9F7099304C
:100B300009F0EBCEE6CEEFE9FFE03197F1F700C028
:100B400000000197009769F3D9CE8DE091E00E94F3
:100B5000C00A982F9F7009F4EBCEF7CEEFE9FFE0C3
:100B60003197F1F700C000000197009771F3DDCED7
:100B7000EFE9FFE03197F1F700C00000019700971F
:100B800009F0FECE8DE091E00E94C40A982F9F707C
:100B9000993009F0FCCEF7CE8DE091E00E94C40AB6
:100BA000982F9F7009F406CF14CFEFE9FFE031973B
:100BB000F1F700C000000197009771F3F8CE88B1FB
:100BC000887F88B98FE99FE00197F1F700C00000A6
:100BD0000F5F1F4F78CDDF91CF911F910F91FF9045
:100BE000EF90DF90CF90BF900895CF92DF92EF9279
:100BF000FF920F931F93CF93DF93809102018F3C5D
:100C000009F0BDC0B1C00C2D1D2D813C49F50E94DD
:100C1000360B80930201882309F49DC016C00E9400
:100C2000360B809302010E949800C536D10514F05E
:100C3000CE2DDF2D8FE99FE00197F1F700C0000076
:100C4000219680910201882351F390E00E94600078
:100C5000682F8DE091E00E94C80A81EC0E942E0B63
:100C600080910201823C49F50E94360B809302017B
:100C7000882309F467C016C00E94360B80930201D6
:100C80000E949800C536D10514F0CE2DDF2D8FE9D6
:100C90009FE00197F1F700C00000219680910201CA
:100CA000882351F390E00E946000682F8DE091E06E
:100CB0000E94CE0A82EC0E942E0B80910201833C9E
:100CC00049F50E94360B80930201882391F116C0EA
:100CD0000E94360B809302010E949800C536D10510
:100CE00014F0CE2DDF2D8FE99FE00197F1F700C0C2
:100CF0000000219680910201882351F390E00E9428
:100D0000600040E0682F8DE091E00E94D40A83ECFF
:100D10000E942E0B80910201843C89F10F5F1F4FCE
:100D20000E94360B80930201053611050CF06BCF43
:100D30006CCF0E94360B809302010E949800CC2D4C
:100D4000DD2DD1CF0E94360B809302010E949800C6
:100D5000CC2DDD2D9CCF0E94360B809302010E948A
:100D60009800CC2DDD2D66CF0E94360B80930201BA
:100D700000E010E0C12CD12CEC2CFD2C46CFDF91F3
:100D8000CF911F910F91FF90EF90DF90CF9008953A
:100D90000F931F938DE091E00E941E0A0BE210E07A
:100DA00025E030E047E050E066E070E083E091E06D
:100DB0000E94DD061F910F9108950F931F93FC0170
:100DC000608371834283538324833583178306832F
:100DD000D8011197B187A0875C9181E090E0FC0178
:100DE00002C0EE0FFF1F2A95E2F79F01252BFC01A1
:100DF00002C0EE0FFF1F4A95E2F7AF01422B02C07F
:100E0000880F991F6A95E2F7842B8C931F910F919D
:100E100008950F931F93CF93DF93FC0180E090E040
:100E200021E030E000E810E070E041113DC0A68113
:100E3000B7815C91E901028002C0CC0FDD1F0A94EA
:100E4000E2F7C095C523CC93DB01082E02C0B5950F
:100E5000A7950A94E2F7A0FF0DC0A681B7815C9127
:100E6000E901008002C0CC0FDD1F0A94E2F7C52B18
:100E7000CC930DC0A681B7815C91E901008002C0CE
:100E8000CC0FDD1F0A94E2F7C095C523CC93A68151
:100E9000B7815C91E901028002C0CC0FDD1F0A948A
:100EA000E2F7C52BCC933EC0A681B7815C91E901E6
:100EB000028002C0CC0FDD1F0A94E2F7C095C52363
:100EC000CC93D801082E02C0B595A7950A94E2F7F5
:100ED000A623B723AB2B69F0A681B7815C91E9010A
:100EE000008002C0CC0FDD1F0A94E2F7C52BCC9323
:100EF0000DC0A681B7815C91E901008002C0CC0FD2
:100F0000DD1F0A94E2F7C095C523CC93A681B78173
:100F10005C91E901028002C0CC0FDD1F0A94E2F768
:100F2000C52BCC9301968830910509F07ECFDF91D7
:100F3000CF911F910F910895FC01A681B7814C912B
:100F400021E030E0C901048002C0880F991F0A9493
:100F5000E2F7842B8C9385E08A95F1F70000A68157
:100F6000B7814C91C901048002C0880F991F0A946F
:100F7000E2F7809584238C930895CF92DF92EF92CD
:100F8000FF920F931F93CF93DF93EC010E94F20A1D
:100F9000CC80DD80EE80FF808B010C191D091F8B3A
:100FA0000E8B043F114020F4CD28CE28CF2871F5B8
:100FB0002D981D8A0E94F20A0C811D812E813F818D
:100FC000AB01BC01401B510B620B730B4C835D8367
:100FD0006E837F830E94F20A688379838A839B836E
:100FE00081E04C815D816E817F81493E5340610586
:100FF000710508F480E0811103C08885882319F009
:1010000081E0888705C01A8A198A02C081E08D8B29
:10101000DF91CF911F910F91FF90EF90DF90CF90D4
:101020000895FC01238934892115310531F46623A3
:1010300009F4F4C040E050E03CC0A901C9010197A7
:10104000439708F4EDC02431310519F46111FCC057
:10105000E9C0C9014597079718F5662381F0C901D2
:10106000459741E050E0BA0102C0660F771F8A95AC
:10107000E2F7CB019385892B838781E0E0C0C9012A
:10108000459741E050E0BA0102C0660F771F8A958C
:10109000E2F7CB01809593858923838781E0CFC0D8
:1010A0002C31310531F4838580FFE0C06111D2C05D
:1010B000BBC0CA014D97069718F5662381F0C90198
:1010C0004D9741E050E0BA0102C0660F771F8A9544
:1010D000E2F7CB019485892B848781E0B0C0C901F8
:1010E0004D9741E050E0BA0102C0660F771F8A9524
:1010F000E2F7CB01809594858923848781E09FC0A6
:101100002332310581F4848580FF09C061110BC051
:101110008DC02332310539F4848580FD04C06623F7
:1011200009F49EC085C0CA018497069718F5662306
:1011300081F0C901849741E050E0BA0102C0660F16
:10114000771F8A95E2F7CB019585892B858781E00A
:1011500076C0C901849741E050E0BA0102C0660F31
:10116000771F8A95E2F7CB0180959585892385873E
:1011700081E065C0CA018A978330910508F45AC09E
:101180000397059718F5662381F0C9018D9741E013
:1011900050E0BA0102C0660F771F8A95E2F7CB01D3
:1011A0009785892B878781E04AC0C9018D9741E0E7
:1011B00050E0BA0102C0660F771F8A95E2F7CB01B3
:1011C000809597858923878781E039C042535109EB
:1011D0004830510588F5662381F0C901C29741E086
:1011E00050E0BA0102C0660F771F8A95E2F7CB0183
:1011F0009089892B808B81E022C0C901C29741E090
:1012000050E0BA0102C0660F771F8A95E2F7CB0162
:10121000809590898923808B81E011C080E00FC088
:1012200081E00DC080E00BC080E009C080E007C015
:1012300080E005C081E003C081E001C080E02F5F55
:101240003F4F348B238B0895C9014597079708F4C6
:1012500006CF0FC0C9014D97069708F42ECF59CF7E
:10126000CA018497069708F474CF84CF662391F35C
:10127000E5CFC9014D97069708F41FCF54CF8F9241
:101280009F92AF92BF92FF920F931F93CF93DF93E2
:10129000EC010E94F20A88809980AA80BB808B01B1
:1012A000081919091F8B0E8B0431110528F48928A0
:1012B0008A288B2809F056C02D9A1D8A0E94F20AAE
:1012C0006C837D838E839F830E94F20A088119813B
:1012D0002A813B81AB01BC01401B510B620B730B9C
:1012E000488359836A837B838885882379F189853C
:1012F0009A85CB977CF581E090E09A8B898BDB0116
:10130000CA0180559109A109B1098997A105B105C3
:1013100050F0445B51096109710949325105610579
:10132000710518F004C0F12C02C0FF24F3946F2D56
:10133000CE010E941108882319F01A861986188692
:1013400089859A8501969A8789870EC089859A85AD
:10135000CB9754F018861A86198682E090E09A8B13
:10136000898B02C081E08D8BDF91CF911F910F910E
:10137000FF90BF90AF909F908F9008951F920F9213
:101380000FB60F9211242F933F934F935F936F9358
:101390007F938F939F93AF93BF93EF93FF93F894B3
:1013A0004A9B05C08FE091E00E943F0904C08FE096
:1013B00091E00E94BD077894FF91EF91BF91AF91AA
:1013C0009F918F917F916F915F914F913F912F915D
:1013D0000F900FBE0F901F90189510920F01109252
:1013E000100110921101109212011092130110922B
:1013F000140110921501109216011092170110920B
:1014000019011092180110921A0110921B011092EA
:101410001C0110921D0110921E0110921F011092CA
:1014200021011092200110922301109222011092AA
:10143000240110922601109225010895FC011182C9
:1014400008958CE58093B800E9EBF0E080818C7F13
:101450008083ECEBF0E084E0808384EA8083808109
:101460008823ECF780ED8093BB0084E88093BC0078
:10147000ECEBF0E080818823ECF76093BB0084E81C
:101480008093BC00ECEBF0E080818823ECF7409384
:10149000BB0084E88093BC00ECEBF0E08081882303
:1014A000ECF784E98093BC00ECEBF0E0808184FDF4
:1014B000FDCFECEBF0E080818B7F808308958CE59D
:1014C0008093B800E9EBF0E080818C7F8083ECEBC7
:1014D000F0E084E0808384EA808380818823ECF7D5
:1014E00080ED8093BB0084E88093BC00ECEBF0E0DF
:1014F00080818823ECF76093BB0084E88093BC0074
:10150000ECEBF0E080818823ECF784EA8093BC0068
:10151000ECEBF0E080818823ECF781ED8093BB0059
:1015200084E88093BC00ECEBF0E080818823ECF74A
:1015300084E88093BC00ECEBF0E080818823ECF73A
:101540008091BB0094E99093BC00ECEBF0E09081BB
:1015500094FDFDCFECEBF0E090819B7F90830895AC
:1015600060E00E945F0A089561E00E945F0A0895AA
:1015700062E00E945F0A089564E00E945F0A089595
:1015800065E00E945F0A089566E00E945F0A089580
:10159000462F60E070E00E94210A0895462F61E026
:1015A00070E00E94210A0895442319F0462F4064F8
:1015B00002C0462F4F7B62E070E00E94210A08952E
:1015C000462F64E070E00E94210A0895462F65E0EE
:1015D00070E00E94210A0895462F66E070E00E94A4
:1015E000210A0895F8946091270170912801809153
:1015F000290190912A01789408951F920F920FB6B5
:101600000F9211248F939F93AF93BF9380912701E3
:1016100090912801A0912901B0912A010196A11D64
:10162000B11D8093270190932801A0932901B093C5
:101630002A01BF91AF919F918F910F900FBE0F9094
:101640001F9018951092C50087E68093C40088E12A
:101650008093C10086E08093C2000895E0ECF0E042
:10166000908195FFFDCF8093C60008958091C000C2
:1016700088231CF48091C600089580E008950E949C
:1016800077000E943E010E944B030E94D9020E94F3
:10169000F505F7CFEE0FFF1F0590F491E02D0994AB
:0416A000F894FFCFEC
:00000001FF
